:020000040000FA
:1000000025006704DF0C02000F0A640C2800F90CBD
:1000100029000000E902090AE802070A00080C0C9E
:100020000600010C26000509090C0600020C26003A
:100030000509090C0600040C260005090C0C060035
:10004000020C260005090A0C0600010C2600050911
:100050000A0C0600040C2600050905090A0C060016
:10006000010C260005090C0C0600020C26000509EF
:10007000090C0600040C26000509090C0600020CF8
:10008000260005090C0C0600010C260005090509CF
:080090000509050905090F0A25
:021FFE00EB0FE7
:00000001FF
